:1000000000308A00622F0000FF00030E8301A10070
:100010000A08A0008A010408A2007708A300780853
:10002000A4007908A5007A08A6007B08A70083131E
:1000300083128B1E1D280B1934288B1D21280B18A9
:100040003728220884002308F7002408F800250830
:10005000F9002608FA002708FB0020088A00210E74
:100060008300FF0E7F0E09008A110A12C8288A1128
:100070000A120A290A108A100A1182073F3406342C
:100080005B344F3466346D347D3407347F346F34E1
:100090000A108A100A118207063454346D345C3415
:1000A000383477345E345C3450347734003473340D
:1000B0005C34503400345E3477345434063479344C
:1000C00038340034BD3400340034FF340A108A1050
:1000D0000A11820739347734383479345434783417
:1000E000773454345E34DC34003477343934393482
:1000F000793473347834773450340034733477344B
:100100005034773400347734393477347C3477346E
:10011000D03400340034FF340A108A100A118207E8
:1001200006340034393477345034F7340034003432
:10013000FF340A108A100A1182075B340034393404
:10014000773450347734ED3400340034FF340A10FF
:100150008A100A118207383406346D347834DC345E
:100160008034803400340034FF340A108A100A11BD
:1001700082076D3479343D343E3454345E34773400
:100180000034393477345034F73400340034FF34D9
:1001900083308100B008031DF0287D30B000AF0827
:1001A0000319D428AF03F028AE080319DB28AE03E7
:1001B0000930AF00F028AD080319E428AD0305307D
:1001C000AE000930AF00F028AC080319EF28AC03EB
:1001D0000930AD000530AE000930AF00F028291419
:1001E000B0030B118A110A122128AE3084000008D6
:1001F000031909290130F800F701F70BFD28F80B66
:10020000FC284A30F700F70B032900000000800BA0
:10021000FA280034861B3A2901303102FC3E0318CB
:100220003329043E80292C08083C031C1929AC0AF8
:100230001A29AC0133292D08083C031C2129AD0AD9
:100240002229AD0133292E08043C031C2929AE0ABA
:100250002A29AE0133292F08083C031C3129AF0A93
:100260003229AF013329861F332932308316AE007D
:100270008312F520061B6A2901303102FC3E031867
:100280006329043E8829AC0803194829AC034A298C
:100290000930AC006329AD0803195029AD03522978
:1002A0000930AD006329AE0803195829AE035A2955
:1002B0000530AE006329AF0803196029AF03622936
:1002C0000930AF006329061F632932308316AE0060
:1002D0008312F520861A7C293108033C031C7229FD
:1002E000B10A74290130B100861A7C293230831694
:1002F000AE008312F52074290B108A110A122128EE
:100300000A148A100A11820713291B2923292B2971
:100310000A148A100A11820743294B2953295B29A1
:10032000630887000514A8018B1BA8178B130230E4
:100330008316AE008312F520A81B8B17051000341E
:10034000630887008514A8018B1BA8178B13023044
:100350008316AE008312F520A81B8B17851000347E
:10036000630887000515A8018B1BA8178B130230A3
:100370008316AE008312F520A81B8B1705110034DD
:10038000630887008515A8018B1BA8178B13023003
:100390008316AE008312F520A81B8B17851100343D
:1003A000DD01DE010130DF000230E0000330E1005A
:1003B00033305D078400000FDE29E029DD0AD829EB
:1003C000AB01AA01AB08031D642A2A085802031CCA
:1003D000642A33305E0784000008E200E3009021C5
:1003E00033305F0784000008E200E300A0213330CF
:1003F000600784000008E200E300B02133306107A9
:1004000084000008E200E300C021861F0D2A061FB9
:100410000D2A861E0D2A061A602A861B242A590BCD
:10042000242A861B162A5A0B162A112AA8018B1B6E
:10043000A8178B1332308316AE008312F520A81B49
:100440008B170030F800852A061B382A5A0B382AE9
:10045000061F282AA8018B1BA8178B13323083167E
:10046000AE008312F520A81B8B170130F800852AF7
:10047000861A4C2A5B0B4C2A861E3C2AA8018B1B31
:10048000A8178B1332308316AE008312F520A81BF9
:100490008B170230F800852A061A602A5C0B602A46
:1004A000061E502AA8018B1BA8178B133230831607
:1004B000AE008312F520A81B8B170330F800852AA5
:1004C000AA0A0319AB0AE22901305D025E02031891
:1004D0006B2ADE0A6C2ADE0101305D025F0203181E
:1004E000732ADF0A742ADF0101305D0260020318FB
:1004F0007B2AE00A7C2AE00101305D0261020318D8
:10050000832AE10A842AE101E0290034D601560851
:100510004820FF3C03198E2AD60A872AAB01AA017C
:10052000AB08031DA42A2A085602031CA42A333050
:100530002A0784002B08FA002A084820F8008000C7
:10054000AA0A0319AB0A902A2330D800D901DA018C
:10055000DB010130DC00D0218A110A129E2FD60166
:10056000851656086620FF3C0319B82AD60AB12A18
:10057000AB01AA01AB08031DCE2A2A085602031CB0
:10058000CE2A33302A0784002B08FA002A08662076
:10059000F8008000AA0A0319AB0ABA2A2330D8004F
:1005A000D901DA010130DB00DC01D02185128A118A
:1005B0000A12A02F561003178D0183168C130C14EA
:1005C00083120C088D0183168C130C1483120C08F3
:1005D000093C031CF42A8D0183168C130C1483121E
:1005E0000C080313AC00031701308D0083168C1325
:1005F0000C1483120C0801308D0083168C130C141C
:1006000083120C08093C031C0F2B01308D0083164C
:100610008C130C1483120C080313AD000317023063
:100620008D0083168C130C1483120C0802308D007D
:1006300083168C130C1483120C08053C031C2A2B04
:1006400002308D0083168C130C1483120C080313D4
:10065000AE00031703308D0083168C130C14831225
:100660000C0803308D0083168C130C1483120C08B5
:10067000093C031C452B03308D0083168C130C148E
:1006800083120C080313AF00031703138B15AB0180
:10069000AA01AB08031D8E2B2A08133C031C8E2BCA
:1006A000310B572B5618572BE30190215C2B2C084C
:1006B0003A20D700E30090213108023C031D662B4D
:1006C0005618662B8030E300A0216C2B2D083A20B1
:1006D000803ED800E300A0213108033C031D752BA8
:1006E0005618752BE301B0217A2B2E083A20D7003B
:1006F000E300B0213108043C031D832B5618832BE3
:10070000E301C021882B2F083A20D700E300C02145
:10071000061E8E2BAA0A0319AB0A492B561C922BD4
:100720005610932B5614061A472B061E952BA8011C
:100730008B1BA8178B1332308316AE008312F52063
:10074000A81B8B178B1103178D0103132C0803179C
:100750008C0083168C130C15831203130B08F700FF
:100760008B138316031755308D00AA308D008C141F
:100770008C18B82B0C117708831203138B040130EB
:1007800003178D0003132D0803178C0083168C1399
:100790000C15831203130B08F7008B138316031732
:1007A00055308D00AA308D008C148C18D52B0C116F
:1007B0007708831203138B04023003178D00031391
:1007C0002E0803178C0083168C130C158312031349
:1007D0000B08F7008B138316031755308D00AA30D2
:1007E0008D008C148C18F22B0C11770883120313D4
:1007F0008B04033003178D0003132F0803178C009D
:1008000083168C130C15831203130B08F7008B133C
:100810008316031755308D00AA308D008C148C1868
:100820000F2C0C117708831203138B048A110A1200
:10083000A12FD601D701320B3A2C57088C20FF3C50
:100840000319242CD70A1D2CAB01AA01AB08031DE8
:100850003A2C2A085702031C3A2C33302A0784000A
:100860002B08FA002A088C20F8008000AA0A031935
:10087000AB0A262C3208023C031D5B2C570899203A
:10088000FF3C0319452CD70A3E2CAB01AA01AB084B
:10089000031D5B2C2A085702031C5B2C33302A07EC
:1008A00084002B08FA002A089920F8008000AA0A80
:1008B0000319AB0A472C2330D8000130D900DA00E5
:1008C000DB00DC01D0217808D600D60803196A2C99
:1008D000560B712C320B6F2C0230B200712C013090
:1008E000B2005608023C0319792C5608033C031D3C
:1008F0001B2C8A110A12A22FD6015608A720FF3CF2
:100900000319842CD60A7D2CAB01AA01AB08031D68
:100910009A2C2A085602031C9A2C33302A0784008A
:100920002B08FA002A08A720F8008000AA0A031959
:10093000AB0A862C2330D800D901DA010130DB0064
:10094000DC01D0218A110A12A32F291003178D016F
:1009500083168C130C1483120C080313AC000130A3
:1009600003178D0083168C130C1483120C080313C9
:10097000AD00023003178D0083168C130C14831204
:100980000C080313AE00033003178D0083168C137D
:100990000C1483120C080313AF00851683308100FA
:1009A0008B16AC080319D92C2C083A20D600E3008A
:1009B0009021AC08031DE32CAD08031DE32C80300F
:1009C000E300A021E92C2D083A20803ED700E30067
:1009D000A0212E083A20D600E300B0212F083A20AB
:1009E000D600E300C021291CD12C8B1285120034C3
:1009F000F701F801F901FA018316A401A501A60186
:100A0000A70123082204210420040319372D2030D4
:100A1000A8000310F20DF30DF40DF50DA40DA50DB6
:100A2000A60DA70D23082702031D202D220826024C
:100A3000031D202D21082502031D202D200824023E
:100A4000031C312D2008A4022108031C210FA5023C
:100A50002208031C220FA6022308031C230FA7024F
:100A60000314F70DF80DF90DFA0DA80B092D000070
:100A7000A430840083120034F801F901F701FA016F
:100A80006C08031D462D6B080319602D1030ED0016
:100A90000310E90DEA0DF70DFA0D6C087A02031D3B
:100AA000532D6B087702031C5C2D6B08F702031CA7
:100AB000FA036C08FA020314F80DF90DED0B482D3A
:100AC0000000003420308316A400A001A101A2017F
:100AD000A3017008FA0083126F08F9006E08F8008D
:100AE0006D08F7000310771C852D71088316A00789
:100AF00072080318720FA10773080318730FA20777
:100B000074080318740FA30783128316A30CA20C96
:100B1000A10CA00CFA0CF90CF80CF70CA40B912DFD
:100B2000932D8312722D83128A110A12722E1230A3
:100B3000EE02031CA92D6E308400FC3080050310EA
:100B4000800C800C00080319A92DA72D0000800B34
:100B5000A62D8A110A12D72DED016A086D0203181D
:100B6000BE2DA8018B1BA8178B13FA308316AE007D
:100B70008312F520A81B8B17ED0AAD2DA8018B1B46
:100B8000A8178B1369088316AE008312F520A81BE3
:100B90008B17ED016C086D020318D42D5330F7004C
:100BA000F70BD02DED0ACA2D6B08EE00972D0034FF
:100BB000F5010F30F4004230F3004030F2008316AC
:100BC000A301A201831258088316A10083125708BB
:100BD0008316A0008312F82403107A0CF000790C1D
:100BE000EF00780CEE00770CED000A306D02DB00B0
:100BF0006E08DC000030031C0130DC026F08DD00F1
:100C00000030031C0130DD027008DE000030031CE0
:100C10000130DE025E08F5005D08F4005C08F300B8
:100C20005B08F2008316A301A2010330A100E830A3
:100C3000A0008312F8247808E0007708DF0060083D
:100C4000EA005F08E900EC01FA30EB003C25780887
:100C5000E4006008EA005F08E900EC01FA30EB000C
:100C60003C257708E5005E08F5005D08F4005C08A7
:100C7000F3005B08F2008316A301A2010330A10078
:100C8000E830A0008312F8240008E100840A00087C
:100C9000E2006208EA006108E900EC01FA30EB00CA
:100CA0003C257808E3006208EA006108E900EC01ED
:100CB000FA30EB003C257708E600EC01EB015A081E
:100CC000EA005908E9006C08F0006B08EF005A08C8
:100CD000EE005908ED00F401F3010330F200E830B2
:100CE000F100622D7A08ED007908EC007808EB003D
:100CF0007708EA00F5010F30F4004230F30040308D
:100D0000F2008316A301A201831258088316A100E2
:100D1000831257088316A0008312F8247A08F10082
:100D20007908F0007808EF007708EE006D08F5000C
:100D30006C08F4006B08F3006A08F2007A08831666
:100D4000A3007908A200831278088316A1008312F9
:100D500077088316A0008312F8247808E800770843
:100D6000E7006808FA0067080319E803E703E900E9
:100D70007A08EA00E908031DC02EEA080319DB2EF1
:100D80006508E9006408EA006608EB006308EC0007
:100D9000AC2583160610831206146508E900640862
:100DA000EA006608EB006308EC00AC258316061029
:100DB00083120610B12E003456100B30D800B83014
:100DC000D700DA016430D900D825861EE92E061A2C
:100DD000FA2E861EED2E061AF92EA8018B1BA817D7
:100DE0008B1332308316AE008312F520A81B8B17AD
:100DF000E92E382F0F30D800A030D700DA01643048
:100E0000D900D825861E062F061A172F861E0A2FF0
:100E1000061A162FA8018B1BA8178B1332308316C6
:100E2000AE008312F520A81B8B17062F382FA801C0
:100E30008B1BA8178B1364308316AE008312F5202A
:100E4000A81B8B17861E262F061A372F861E2A2FC1
:100E5000061A362FA8018B1BA8178B133230831666
:100E6000AE008312F520A81B8B17262F382FDD2EFE
:100E70000034D6015608B520FF3C0319412FD60A8D
:100E80003A2FAB01AA01AB08031D572F2A085602BF
:100E9000031C572F33302A0784002B08FA002A0836
:100EA000B520F8008000AA0A0319AB0A432F2330AB
:100EB000D800D901DA010130DB00DC01D0218A1130
:100EC0000A12AA2F84011F30830583161F149F1452
:100ED0001F159F118312AC01AD01AE01AF017D3032
:100EE000B0000130B100B2000030831685008113DC
:100EF000FC3086000030870083128501860187015F
:100F00000530F700F71D8C2F0730810181308400F8
:100F10000008C0390F388000640081308400000868
:100F2000C039770480007830F80006389200FF302E
:100F300083169200C03083128B04862A8614AF2A4F
:100F4000DA2A192C7C2CA524DC263208023C031D4D
:100F5000AC2F392FA524DC2686108A0100286300D7
:02400E00313F40
:00000001FF
